:1000000019C0CFC132C031C030C02FC030C12DC0E7
:100010002CC02CC02AC029C028C027C026C025C09B
:1000200030C0F7C106C209C208C245C244C266C296
:10003000F2C101C211241FBECFE5D1E0DEBFCDBFAA
:1000400010E0A0E6B0E0E2E0F6E002C005900D921C
:10005000A236B107D9F710E0A2E6B0E001C01D92C8
:10006000A839B107E1F7C5D0CAC2CACF1F920F9213
:100070000FB60F921124689A0F900FBE0F901F9029
:1000800018951F920F920FB60F9211248F938091A3
:10009000970080FF03C089B78D7F89BF80E48EB948
:1000A000809197008260809397008FB18093960033
:1000B0008F910F900FBE0F901F9018959AB3906379
:1000C0009ABBD698DE9A880F880F8A658DB983E02F
:1000D00083BF81E086BF8091970081608093970005
:1000E000809197008D7F80939700809197008B7F00
:1000F00080939700109296000895D59AD6989BB356
:1001000090659BBB880F880F88658DB9809197009B
:100110008E7F80939700809197008D7F80939700CA
:10012000809197008B7F809397001092960008959E
:100130002EB130E02F7030702115310539F08091EB
:10014000970084608093970080E0089590919700D5
:100150009D7F90939700909197009B7F909397003D
:100160008FB98091970080FF06C088B7826088BFF2
:1001700089B7826089BF9091970081E092FD80E00D
:1001800008958091960008958091970081FFFCCF9B
:100190000895D198D398B99AC198D698089582E0D5
:1001A00085BF8BB780648BBFBA98C29A6E986C98E3
:1001B00008958EB582608EBD8EB588608EBD88EC48
:1001C00090E09BBD8ABD619A08950098379A86B1E8
:1001D000866086B917B83F983E9A0895F8941092B1
:1001E000800010929500D5DFF0DFD9DFE2DF789450
:1001F00008958FEF92E0880F991FC3D1909361000B
:1002000080936000EBDFFFCF97B1907E97B997B1F5
:100210008F71892B87B9369A3699FECF84B195B103
:10022000392F20E0280F311DC9010895623059F49B
:10023000282F392FD901ECE6F0E025E101900D924D
:100240002150E1F70895282F392FD901E1E8F0E096
:1002500025E101900D922150E1F70895843019F4C1
:1002600024E630E002C028E630E0C90108951F927C
:100270000F920FB60F9211241F932F933F934F931A
:100280005F936F937F938F939F93AF93BF93CF931E
:10029000DF93EF93FF9310918000C12FD0E083E0B4
:1002A000B3DFCC0FDD1FC459DF4F998388831F5FF5
:1002B0001093800080916400909165000097F1F0A8
:1002C000E0918000F0E0EE0FFF1FE659FF4F208124
:1002D000318180916400909165002817390770F092
:1002E000E0918000F0E0EE0FFF1FE659FF4F8081A4
:1002F00091819093670080936600C19A80918000FD
:100300008A3011F41092800010919500C12FD0E036
:1003100081E07ADFCC0FDD1FCF57DF4F99838883D1
:100320001F5F10939500809168009091690000977D
:10033000F1F0E0919500F0E0EE0FFF1FE158FF4F64
:1003400020813181809168009091690028173907D8
:1003500070F0E0919500F0E0EE0FFF1FE158FF4FC5
:100360008081918190936B0080936A00C19A809103
:1003700095008A3011F410929500FF91EF91DF9172
:10038000CF91BF91AF919F918F917F916F915F912D
:100390004F913F912F911F910F900FBE0F901F9083
:1003A00018951F920F920FB60F921124DF92EF92C1
:1003B000FF920F931F932F933F934F935F936F93EE
:1003C0007F938F939F93AF93BF93EF93FF93DF93AD
:1003D000CF93CDB7DEB76897DEBFCDBF619880E021
:1003E0008CDE78948DB180658DB985E5A1DECCDE9B
:1003F0000091960019821B821A82802F99DEC4DE3A
:10040000E02FF0E0E930F10508F09BC0EF5EFF4F10
:10041000099483E30BC08091600090916100892F63
:1004200087DEB2DE809160009091610081DEACDEFB
:1004300088C0D9D0FBCFD3D0F9CFCE010496602F9E
:10044000F5DE809196008983898172DE9DDE1092AF
:10045000630010926200B9E0DB2E7E010894E11C7B
:10046000F11C1EC0888D882309F4D88E888D815098
:10047000888FE88DF0E0EE0FFF1FEE0DFF1D03816A
:100480001481812F55DE80DE802F52DE7DDE80914B
:1004900062009091630001969093630080936200E4
:1004A0002091620030916300898190E0281739071C
:1004B000CCF286E1BBCF3091960020E03B832A83CB
:1004C0002A813B81832F34DE5FDE4A815B8120916C
:1004D000960030E0242B352B3B832A838A819B8135
:1004E00027DE52DE043019F4E4E6F0E002C0E8E66C
:1004F000F0E08A819B819183808323C08091660094
:1005000090916700892F14DE3FDE80916600909104
:1005100067000EDE39DE109267001092660080914F
:100520006A0090916B00892F03DE2EDE80916A00B5
:1005300090916B00FDDD28DE10926B0010926A0036
:10054000C1986E986C98D698D598619A6896DEBFD7
:10055000CDBFCF91DF91FF91EF91BF91AF919F916F
:100560008F917F916F915F914F913F912F911F914B
:100570000F91FF90EF90DF900F900FBE0F901F90A4
:100580001895CF93009731F140E050E02FEF3FEF07
:1005900068E074E8FA014F5F5F4FE491F0E0C8E073
:1005A000D901AE27BF2736952795A0FF02C0262781
:1005B0003727C15019F0F695E795F2CF481759073C
:1005C00049F720953095922F8827232F3327282B02
:1005D000392B02C020E030E0C901CF91089580E0BE
:1005E00090E005D0089581E090E001D00895E19970
:1005F000FECF1FBA8EBBE09A99278DB30895F89469
:02060000FFCF2A
:02060200FFFFF8
:00000001FF
